:1000000000308A005F280000FF00030E8301A60075
:100010007F08A5000A08AD008A01A50E0408A70004
:100020002008A8002108A9002208AA002308AB0084
:100030002408AC00831383128B1E20280B1933284D
:10004000270884002808A0002908A1002A08A20087
:100050002B08A3002C08A4002D088A00260E83007C
:10006000FF0E7F0E09008A11352830088100B10B80
:1000700046283230B100831685168312851E422829
:100080008512432885168316851283120B118A1157
:10009000202833308400000803195D280330A100B4
:1000A000A001A00B5128A10B50283C30A000A00BB0
:1000B000572800000000800B4E288A117E298401F9
:1000C0001F30830583161F149F141F159F11FF30C7
:1000D0008312B2003230B10032103208831687002A
:1000E00083120714B2113208831687008312871512
:1000F0000130831685000030860087008312B2002D
:100100003211320883168700831207110C309700D2
:10011000B210320883168700831287100C309D00BE
:100120000030A10004389200FF30831692001F10A7
:100130009F141F159F1583121F139F1783169F1758
:1001400083121F1483160108C039073881008312F7
:1001500081018B16C0308B040030A1001F08C73905
:1001600021049F001030A000A00BB42800001F1530
:100170001F19B82883161E088312AE001E08AF0090
:100180002F08013C03180C29FF3A031DCB282E0829
:10019000103C03180C293210320883168700831292
:1001A0000714B211320883168700831287150030B6
:1001B0002E02A0002F08A3000230031C0330A3026C
:1001C0002008A2000310200DB300230DB400B40CCE
:1001D000B30CB40CB30CB40C33089B00B40C340C4B
:1001E0003039A0001D08CF3920049D009501B211BF
:1001F0003208831687008312871100302E02B30065
:100200002F08B4000230031C0330B4020310340C76
:10021000A300330CA200B0002F08013C031C572997
:10022000031D16292E08EF3C031C572932103208F3
:100230008316870083120714B211320883168700D1
:10024000831287159B012E08FF3CA0000130A300FC
:100250002F08031C2F0FA3022008A2000310200D5B
:10026000B300230DB400B40CB30CB40CB30CB40C39
:1002700033089500B40C340C3039A0001708CF397E
:10028000200497003210320883168700831207106B
:100290002E08FF3CB3000130B4002F08031C2F0FC1
:1002A000B4020310340CA300330CA200B0002F08DA
:1002B000003C03187B29FF3A031D62292E08EF3CFE
:1002C00003187B292F08023C031C7B29031D6C2982
:1002D0002E08103C031C7B2932103208831687003D
:1002E00083120714B2113208831687008312871510
:1002F00095019B01B0011430B3004928AC2863007C
:02400E00723FFF
:00000001FF
